

Microchip Technology PIC18 LITE Macro Assembler V1.37 build -260352376 
                                                                                               Wed Sep 21 21:45:18 2016

Microchip Technology Omniscient Code Generator v1.37 (Free mode) build 201603110536
     1                           	processor	18F4550
     2                           	fnconf	rparam,??,?,0
     3                           	opt	pw 120
     4                           	opt	lm
     5                           	psect	cinit,global,reloc=2,class=CODE,delta=1
     6                           	psect	cstackCOMRAM,global,class=COMRAM,space=1,delta=1
     7                           	psect	text0,global,reloc=2,class=CODE,delta=1
     8                           	psect	text1,global,reloc=2,class=CODE,delta=1
     9                           	psect	intsave_regs,global,class=BIGRAM,space=1,delta=1
    10                           	psect	rparam,global,class=COMRAM,space=1,delta=1
    11  0000                     _CCP1CON	set	4029
    12  0000                     _CCP2CON	set	4026
    13  0000                     _CCPR1L	set	4030
    14  0000                     _CCPR2L	set	4027
    15  0000                     _LATD	set	3980
    16  0000                     _PORTC	set	3970
    17  0000                     _PORTD	set	3971
    18  0000                     _PR2	set	4043
    19  0000                     _T2CON	set	4042
    20  0000                     _TRISC	set	3988
    21  0000                     _TRISD	set	3989
    22                           
    23                           ; #config settings
    24  0000                     
    25                           	psect	cinit
    26  007F40                     __pcinit:
    27                           	opt stack 0
    28  007F40                     start_initialization:
    29                           	opt stack 0
    30  007F40                     __initialization:
    31                           	opt stack 0
    32  007F40                     end_of_initialization:
    33                           	opt stack 0
    34  007F40                     __end_of__initialization:
    35                           	opt stack 0
    36  007F40  0100               	movlb	0
    37  007F42  EFBE  F03F         	goto	_main	;jump to C main() function
    38                           
    39                           	psect	cstackCOMRAM
    40  000001                     __pcstackCOMRAM:
    41                           	opt stack 0
    42  000001                     delay_ms@n:
    43                           	opt stack 0
    44                           
    45                           ; 4 bytes @ 0x0
    46  000001                     	ds	4
    47  000005                     ??_delay_ms:
    48                           
    49                           ; 1 bytes @ 0x4
    50  000005                     	ds	1
    51  000006                     main@dc:
    52                           	opt stack 0
    53                           
    54                           ; 1 bytes @ 0x5
    55  000006                     	ds	1
    56                           
    57 ;;
    58 ;;Main: autosize = 0, tempsize = 0, incstack = 0, save=0
    59 ;;
    60 ;; *************** function _main *****************
    61 ;; Defined at:
    62 ;;		line 21 in file "main_PWM.c"
    63 ;; Parameters:    Size  Location     Type
    64 ;;		None
    65 ;; Auto vars:     Size  Location     Type
    66 ;;  dc              1    5[COMRAM] unsigned char 
    67 ;; Return value:  Size  Location     Type
    68 ;;                  1    wreg      void 
    69 ;; Registers used:
    70 ;;		wreg, status,2, status,0, cstack
    71 ;; Tracked objects:
    72 ;;		On entry : 0/0
    73 ;;		On exit  : 0/0
    74 ;;		Unchanged: 0/0
    75 ;; Data sizes:     COMRAM   BANK0   BANK1   BANK2   BANK3   BANK4   BANK5   BANK6   BANK7
    76 ;;      Params:         0       0       0       0       0       0       0       0       0
    77 ;;      Locals:         1       0       0       0       0       0       0       0       0
    78 ;;      Temps:          0       0       0       0       0       0       0       0       0
    79 ;;      Totals:         1       0       0       0       0       0       0       0       0
    80 ;;Total ram usage:        1 bytes
    81 ;; Hardware stack levels required when called:    1
    82 ;; This function calls:
    83 ;;		_delay_ms
    84 ;; This function is called by:
    85 ;;		Startup code after reset
    86 ;; This function uses a non-reentrant model
    87 ;;
    88                           
    89                           	psect	text0
    90  007F7C                     __ptext0:
    91                           	opt stack 0
    92  007F7C                     _main:
    93                           	opt stack 30
    94                           
    95                           ;main_PWM.c: 22: unsigned char dc;
    96                           ;main_PWM.c: 23: TRISC = 0;
    97                           
    98                           ;incstack = 0
    99  007F7C  0E00               	movlw	0
   100  007F7E  6E94               	movwf	3988,c	;volatile
   101                           
   102                           ;main_PWM.c: 24: PORTC = 0;
   103  007F80  0E00               	movlw	0
   104  007F82  6E82               	movwf	3970,c	;volatile
   105                           
   106                           ;main_PWM.c: 25: TRISD = 0;
   107  007F84  0E00               	movlw	0
   108  007F86  6E95               	movwf	3989,c	;volatile
   109                           
   110                           ;main_PWM.c: 26: PORTD = 0;
   111  007F88  0E00               	movlw	0
   112  007F8A  6E83               	movwf	3971,c	;volatile
   113                           
   114                           ;main_PWM.c: 30: PR2 = 0b11111111;
   115  007F8C  68CB               	setf	4043,c	;volatile
   116                           
   117                           ;main_PWM.c: 32: T2CON = 0b00000111;
   118  007F8E  0E07               	movlw	7
   119  007F90  6ECA               	movwf	4042,c	;volatile
   120                           
   121                           ;main_PWM.c: 34: CCP1CON = 0b00111100;
   122  007F92  0E3C               	movlw	60
   123  007F94  6EBD               	movwf	4029,c	;volatile
   124                           
   125                           ;main_PWM.c: 40: CCP2CON = 0b00111100;
   126  007F96  0E3C               	movlw	60
   127  007F98  6EBA               	movwf	4026,c	;volatile
   128  007F9A                     l33:
   129                           
   130                           ;main_PWM.c: 47: for (dc = 0; dc < 128; dc++) {
   131  007F9A  0E00               	movlw	0
   132  007F9C  6E06               	movwf	main@dc,c
   133  007F9E                     l682:
   134  007F9E  0E7F               	movlw	127
   135  007FA0  6406               	cpfsgt	main@dc,c
   136  007FA2  D001               	goto	l34
   137  007FA4  D014               	goto	l694
   138  007FA6                     l34:
   139                           
   140                           ;main_PWM.c: 48: LATD = dc;
   141  007FA6  C006  FF8C         	movff	main@dc,3980	;volatile
   142                           
   143                           ;main_PWM.c: 49: CCPR1L = dc;
   144  007FAA  C006  FFBE         	movff	main@dc,4030	;volatile
   145                           
   146                           ;main_PWM.c: 51: CCPR2L = 128 - dc;
   147  007FAE  5006               	movf	main@dc,w,c
   148  007FB0  0800               	sublw	0
   149  007FB2  0F80               	addlw	128
   150  007FB4  6EBB               	movwf	4027,c	;volatile
   151                           
   152                           ;main_PWM.c: 52: delay_ms(100);
   153  007FB6  0E64               	movlw	100
   154  007FB8  6E01               	movwf	delay_ms@n,c
   155  007FBA  0E00               	movlw	0
   156  007FBC  6E02               	movwf	delay_ms@n+1,c
   157  007FBE  0E00               	movlw	0
   158  007FC0  6E03               	movwf	delay_ms@n+2,c
   159  007FC2  0E00               	movlw	0
   160  007FC4  6E04               	movwf	delay_ms@n+3,c
   161  007FC6  ECA3  F03F         	call	_delay_ms	;wreg free
   162  007FCA  2A06               	incf	main@dc,f,c
   163  007FCC  D7E8               	goto	l682
   164  007FCE                     l694:
   165                           
   166                           ;main_PWM.c: 53: }
   167                           ;main_PWM.c: 54: for (dc = 127; dc > 0; dc--) {
   168  007FCE  0E7F               	movlw	127
   169  007FD0  6E06               	movwf	main@dc,c
   170  007FD2  5006               	movf	main@dc,w,c
   171  007FD4  B4D8               	btfsc	status,2,c
   172  007FD6  D7E1               	goto	l33
   173                           
   174                           ;main_PWM.c: 55: LATD = dc;
   175  007FD8  C006  FF8C         	movff	main@dc,3980	;volatile
   176                           
   177                           ;main_PWM.c: 56: CCPR1L = dc;
   178  007FDC  C006  FFBE         	movff	main@dc,4030	;volatile
   179                           
   180                           ;main_PWM.c: 57: CCPR2L = 128 - dc;
   181  007FE0  5006               	movf	main@dc,w,c
   182  007FE2  0800               	sublw	0
   183  007FE4  0F80               	addlw	128
   184  007FE6  6EBB               	movwf	4027,c	;volatile
   185                           
   186                           ;main_PWM.c: 58: delay_ms(100);
   187  007FE8  0E64               	movlw	100
   188  007FEA  6E01               	movwf	delay_ms@n,c
   189  007FEC  0E00               	movlw	0
   190  007FEE  6E02               	movwf	delay_ms@n+1,c
   191  007FF0  0E00               	movlw	0
   192  007FF2  6E03               	movwf	delay_ms@n+2,c
   193  007FF4  0E00               	movlw	0
   194  007FF6  6E04               	movwf	delay_ms@n+3,c
   195  007FF8  ECA3  F03F         	call	_delay_ms	;wreg free
   196  007FFC  0606               	decf	main@dc,f,c
   197  007FFE  D7E9               	goto	L1
   198  008000                     __end_of_main:
   199                           	opt stack 0
   200                           status	equ	0xFD8
   201                           
   202 ;; *************** function _delay_ms *****************
   203 ;; Defined at:
   204 ;;		line 146 in file "Alteri.h"
   205 ;; Parameters:    Size  Location     Type
   206 ;;  n               4    0[COMRAM] long 
   207 ;; Auto vars:     Size  Location     Type
   208 ;;		None
   209 ;; Return value:  Size  Location     Type
   210 ;;                  1    wreg      void 
   211 ;; Registers used:
   212 ;;		wreg, status,2, status,0
   213 ;; Tracked objects:
   214 ;;		On entry : 0/0
   215 ;;		On exit  : 0/0
   216 ;;		Unchanged: 0/0
   217 ;; Data sizes:     COMRAM   BANK0   BANK1   BANK2   BANK3   BANK4   BANK5   BANK6   BANK7
   218 ;;      Params:         4       0       0       0       0       0       0       0       0
   219 ;;      Locals:         0       0       0       0       0       0       0       0       0
   220 ;;      Temps:          1       0       0       0       0       0       0       0       0
   221 ;;      Totals:         5       0       0       0       0       0       0       0       0
   222 ;;Total ram usage:        5 bytes
   223 ;; Hardware stack levels used:    1
   224 ;; This function calls:
   225 ;;		Nothing
   226 ;; This function is called by:
   227 ;;		_main
   228 ;; This function uses a non-reentrant model
   229 ;;
   230                           
   231                           	psect	text1
   232  007F46                     __ptext1:
   233                           	opt stack 0
   234  007F46                     _delay_ms:
   235                           	opt stack 30
   236                           
   237                           ;Alteri.h: 148: while(n-- !=0){
   238                           
   239                           ;incstack = 0
   240  007F46  D008               	goto	l676
   241  007F48                     l674:
   242                           
   243                           ;Alteri.h: 149: _delay((unsigned long)((1)*(48000000/4000.0)));
   244  007F48  0E10               	movlw	16
   245  007F4A  6E05               	movwf	??_delay_ms& (0+255),c
   246  007F4C  0E94               	movlw	148
   247  007F4E                     u117:
   248  007F4E  2EE8               	decfsz	wreg,f,c
   249  007F50  D7FE               	goto	u117
   250  007F52  2E05               	decfsz	??_delay_ms& (0+255),f,c
   251  007F54  D7FC               	goto	u117
   252  007F56  D000               	nop2	
   253  007F58                     l676:
   254  007F58  0EFF               	movlw	255
   255  007F5A  2601               	addwf	delay_ms@n,f,c
   256  007F5C  0EFF               	movlw	255
   257  007F5E  2202               	addwfc	delay_ms@n+1,f,c
   258  007F60  0EFF               	movlw	255
   259  007F62  2203               	addwfc	delay_ms@n+2,f,c
   260  007F64  0EFF               	movlw	255
   261  007F66  2204               	addwfc	delay_ms@n+3,f,c
   262  007F68  2801               	incf	delay_ms@n,w,c
   263  007F6A  E1EE               	bnz	l674
   264  007F6C  2802               	incf	delay_ms@n+1,w,c
   265  007F6E  E1EC               	bnz	l674
   266  007F70  2803               	incf	delay_ms@n+2,w,c
   267  007F72  E1EA               	bnz	l674
   268  007F74  2804               	incf	delay_ms@n+3,w,c
   269  007F76  B4D8               	btfsc	status,2,c
   270  007F78  0012               	return	
   271  007F7A  D7E6               	goto	l674
   272  007F7C                     __end_of_delay_ms:
   273                           	opt stack 0
   274  0000                     wreg	equ	0xFE8
   275                           status	equ	0xFD8
   276                           wreg	equ	0xFE8
   277                           status	equ	0xFD8
   278                           
   279                           	psect	rparam
   280  0000                     wreg	equ	0xFE8
   281                           status	equ	0xFD8


Data Sizes:
    Strings     0
    Constant    0
    Data        0
    BSS         0
    Persistent  0
    Stack       0

Auto Spaces:
    Space          Size  Autos    Used
    COMRAM           95      6       6
    BANK0           160      0       0
    BANK1           256      0       0
    BANK2           256      0       0
    BANK3           256      0       0
    BANK4           256      0       0
    BANK5           256      0       0
    BANK6           256      0       0
    BANK7           256      0       0

Pointer List with Targets:

    None.

Critical Paths under _main in COMRAM

    _main->_delay_ms

Critical Paths under _main in BANK0

    None.

Critical Paths under _main in BANK1

    None.

Critical Paths under _main in BANK2

    None.

Critical Paths under _main in BANK3

    None.

Critical Paths under _main in BANK4

    None.

Critical Paths under _main in BANK5

    None.

Critical Paths under _main in BANK6

    None.

Critical Paths under _main in BANK7

    None.

Call Graph Tables:

 ---------------------------------------------------------------------------------
 (Depth) Function   	        Calls       Base Space   Used Autos Params    Refs
 ---------------------------------------------------------------------------------
 (0) _main                                                 1     1      0     332
                                              5 COMRAM     1     1      0
                           _delay_ms
 ---------------------------------------------------------------------------------
 (1) _delay_ms                                             5     1      4     108
                                              0 COMRAM     5     1      4
 ---------------------------------------------------------------------------------
 Estimated maximum stack depth 1
 ---------------------------------------------------------------------------------

 Call Graph Graphs:

 _main (ROOT)
   _delay_ms

 Address spaces:
Name               Size   Autos  Total    Cost      Usage
BITCOMRAM           5F      0       0       0        0.0%
EEDATA             100      0       0       0        0.0%
NULL                 0      0       0       0        0.0%
CODE                 0      0       0       0        0.0%
COMRAM              5F      6       6       1        6.3%
STACK                0      0       0       2        0.0%
DATA                 0      0       0       3        0.0%
BITBANK0            A0      0       0       4        0.0%
BANK0               A0      0       0       5        0.0%
BITBANK1           100      0       0       6        0.0%
BANK1              100      0       0       7        0.0%
BITBANK2           100      0       0       8        0.0%
BANK2              100      0       0       9        0.0%
BITBANK3           100      0       0      10        0.0%
BANK3              100      0       0      11        0.0%
BITBANK4           100      0       0      12        0.0%
BANK4              100      0       0      13        0.0%
BITBANK5           100      0       0      14        0.0%
BANK5              100      0       0      15        0.0%
BITBANK6           100      0       0      16        0.0%
BANK6              100      0       0      17        0.0%
BITBANK7           100      0       0      18        0.0%
BANK7              100      0       0      19        0.0%
ABS                  0      0       0      20        0.0%
BIGRAM             7FF      0       0      21        0.0%
BITSFR               0      0       0      40        0.0%
SFR                  0      0       0      40        0.0%


Microchip Technology PIC18 Macro Assembler V1.37 build -260352376 
Symbol Table                                                                                   Wed Sep 21 21:45:18 2016

                     l33 7F9A                       l34 7FA6              __CFG_BOR$ON 000000  
            __CFG_BORV$3 000000             __CFG_CP0$OFF 000000             __CFG_CP1$OFF 000000  
                    l674 7F48                      l682 7F9E                      l676 7F58  
                    l694 7FCE             __CFG_CPB$OFF 000000                      u117 7F4E  
                    _PR2 000FCB                      wreg 000FE8             __CFG_LVP$OFF 000000  
           __CFG_WDT$OFF 000000                     _LATD 000F8C                     _main 7F7C  
                   start 1000            __CFG_IESO$OFF 000000            __CFG_MCLRE$ON 000000  
           ___param_bank 000010            __CFG_PLLDIV$5 000000                    ?_main 0001  
                  _T2CON 000FCA                    _PORTC 000F82                    _PORTD 000F83  
          __CFG_USBDIV$2 000000                    _TRISC 000F94                    _TRISD 000F95  
          __CFG_PWRT$OFF 000000            __CFG_WRT0$OFF 000000            __CFG_WRT1$OFF 000000  
         __CFG_EBTR0$OFF 000000           __CFG_FCMEN$OFF 000000           __CFG_EBTR1$OFF 000000  
          __CFG_WRTB$OFF 000000            __CFG_WRTC$OFF 000000           __CFG_EBTRB$OFF 000000  
                  status 000FD8          __initialization 7F40             __end_of_main 8000  
                 ??_main 0006            __activetblptr 000000                   _CCPR1L 000FBE  
                 _CCPR2L 000FBB           __CFG_VREGEN$ON 000000         __end_of_delay_ms 7F7C  
         __CFG_XINST$OFF 000000           __CFG_STVREN$ON 000000                   main@dc 0006  
             __accesstop 0060  __end_of__initialization 7F40          __CFG_PBADEN$OFF 000000  
          ___rparam_used 000001           __pcstackCOMRAM 0001                  _CCP1CON 000FBD  
                _CCP2CON 000FBA                ?_delay_ms 0001                  __Hparam 0000  
                __Lparam 0000                  __pcinit 7F40                  __ramtop 0800  
                __ptext0 7F7C                  __ptext1 7F46               ??_delay_ms 0005  
   end_of_initialization 7F40      start_initialization 7F40         __CFG_LPT1OSC$OFF 000000  
      __size_of_delay_ms 0036                delay_ms@n 0001         __CFG_WDTPS$32768 000000  
               __Hrparam 0000                 __Lrparam 0000                 _delay_ms 7F46  
          __size_of_main 0084    __CFG_CPUDIV$OSC1_PLL2 000000       __CFG_FOSC$HSPLL_HS 000000  
